:1000000000308A00E52900000A108A100A118207D0
:10001000003400340634403420340134FF343F349B
:10002000ED3409342D341234DB34243400340134FB
:100030003134003407340034C0343F34C034093420
:1000400000341034C03400340034403400341234EE
:100050003F34123400340934DB3400348F3400343C
:10006000E634003469340434FD340034013412348D
:10007000FF340034E734003400341C3400342334BB
:1000800000340634C834003400343034A334083427
:10009000BB340134F7340034BF3400343934003415
:1000A000DE3400347934003471340034BD3400342B
:1000B000F6340034093409341E3400347034063404
:1000C0003834003436342234363424343F34003467
:1000D000F33400343F340434F3340434ED34003466
:1000E000013409343E34003430341234363414349C
:1000F0000034363400342A34093412346034003485
:10010000003424348234003400342234083400347F
:1001100000342034F7340034BF3400343934003430
:10012000DE3400347934003471340034BD340034AA
:10013000F6340034093409341E3400347034063483
:100140003834003436342234363424343F340034E6
:10015000F33400343F340434F3340434ED340034E5
:10016000013409343E34003430341234363414341B
:100170000034363400342A3409341234403406341E
:100180000034093480343034C03412340A108A10F8
:100190000A11820747346F34743420347634613462
:1001A0006C343A3420343034783425344C34583478
:1001B0000A340D3400340A108A100A1182075234AE
:1001C0006534613464347934203474346F342034C9
:1001D00064346934733470346C34613479342E345B
:1001E0000A340D340034A0132008831687008312CC
:1001F00087130830F800000000000000F8170F29EE
:10020000F813A80C03188717031C871378170F29F6
:100210007813F80B01290000000000008717A730B1
:100220008400840B11290000F81B0029781B082981
:1002300000340830F7002017200883168700831247
:10024000071B2029A401F7173329F71333290310BB
:10025000071B0314A40C771733297713F70B2729EF
:100260002408F8003F29A730F71B2D30F800F80BC1
:1002700037290000F71B2529771B2D2927298A11EB
:100280000A12172AA71B54290F30F700260EF7056C
:100290000A30770203184F293030F7075129270811
:1002A000F7077708A800F3200F30A6050A302602CA
:1002B00003185C2930305E29A7132708A6072608F3
:1002C000A800F320003494138C112D089300023001
:1002D000941B71298C1D6A2900308316111B013073
:1002E0008312F80000348D119413831611148312B5
:1002F0008D197329941B7329831611187D29831274
:100300002B08AD0063212C08AD0063218316111565
:1003100011198829831200342408A50025081F3CE0
:100320000318A62925087E3C031CA6292030A50217
:100330000310250DF700A600260A0420FA0026085F
:100340000420F8007A08F900A929A9290030F8004A
:10035000F9007908A3007808A200A5012508C620A5
:10036000A50AA800F3200B302502031DAE2923089F
:10037000A6003730A70042212208A6003730A70088
:1003800042210A30A800F3200D30A800F3202308F2
:10039000A6002208A5002508FF3AA7002608A80005
:1003A0004030AB002708AC0073212608A700A80145
:1003B0002608FF3AA9002808AA004230AB00290805
:1003C000AC0073218A110A12332A84011F3083057D
:1003D000073083169F00FF308312A000A01320086F
:1003E0008316870083128717A015200883168700BD
:1003F000831220162008831687003130930028309E
:10040000831294008316941714130912860188012D
:10041000FF30831286008800A4012408DB20A40A90
:10042000A800F32013302402031D0D2A192978088F
:10043000A1002108A800F3202030A800F3203D30BF
:10044000A800F3202030A800F3202108A6003730B0
:10045000A70042210A30A800F3200D30A800F320A5
:0A0460002108A4008C29162A63006D
:02400E007A3FF7
:00000001FF
